:100000000C94460018950000189500001895000003
:10001000189500001895000018950000189500002C
:10002000189500001895000018950000189500001C
:10003000189500001895000018950000189500000C
:100040000C9478231895000018950000189500006E
:1000500018950000189500001895000018950000EC
:1000600018950000189500001895000018950000DC
:1000700018950000189500001895000018950000CC
:100080001895000018950000189500008FEF8DBF9F
:10009000C0E8E4E54E2E80E18EBFD0E1FFE05F2EA8
:1000A000EEEFFFE0A0E0B1E0A89584B7082E877FCF
:1000B00084BF88E1992781BD91BD88278D933197B1
:1000C000E9F785E089B980E08093900088E18AB9FA
:1000D00066248CEF84BB0E94A01A789488E080BFCD
:1000E00085E083BF87B7816087BFBE9A81E28FBDFD
:1000F00081E08EBD86E886B980E087B9B89AC09A5B
:10010000B89AC09A0E94971981E090E00E94A619BF
:10011000BC98BD9A89988C9A8D9A8E9A8F9A1298CB
:10012000139814981598179A00E014E827ED37E112
:10013000A6EDB9E00D931D932D933C930E94E5002D
:100140000E940A010E948C0D0E94930D00E01EEA9D
:100150002DEA38E0A2EDB9E00D931D932D933C9369
:1001600000EE1BEB2EE931E0A2EDB9E00D931D93FB
:100170002D933C93E2EDF9E0FA93EA930E94110F7C
:100180002296E3EBF9E0FA93EA930E949C0F229601
:100190000E947D0A0027A0E3B0E08C9181FB0EF461
:1001A00001E040E0041711F00C94DA001F9A0E945D
:1001B0007D0A1F980E94AB040E944D020E94B0036A
:1001C0000E9489011F980C9400001A9A1C9A1D9A8B
:1001D0001B9AC49A919A969895989498979880E0CB
:1001E0008093B2091F98ACE0B1E0E4E8FCE40E941F
:1001F0005A230E9423200E94FC1BA5E1B1E0EEE8F7
:10020000FCE40E945A230E9423200E94021C0E94A8
:10021000FB1A08950027A0E3B0E08C9181FB0EF457
:1002200001E041E0041711F00C94640180E693E1D1
:10023000A1E0B1E08D939C9382E08093030181E083
:1002400080930401882780930501E8E9FCE40E947B
:100250005A230E94851985E08093030180E18093F1
:100260000401882780930501E2EAFCE40E945A23F6
:100270000E94851980E08093B2090091B2090F3F76
:1002800018F011F00C945D01A2EBB9E08C91992764
:100290009093490080934800A2EBB9E08C918F5F66
:1002A0008C9388E090E00E94A619A2EBB9E08C91B3
:1002B0008F5F8C9310F40C943D010E94FB1A1F9ADF
:1002C0000E9408020C94880180E693E1A1E0B1E06D
:1002D0008D939C9382E08093030181E080930401DD
:1002E000882780930501EAEAFCE40E945A230E94D1
:1002F000851985E08093030188E1809304018827B4
:1003000080930501E4EBFCE40E945A230E948519C6
:1003100008950E94FB1A82EE9FE0A1E0B1E08D9368
:100320009C9381E0E3E30E94DF22AAEDB9E0E7EECF
:10033000F9E098E00E94AA2481E08093E20900910C
:10034000E209083018F011F00C94C701A2EEB9E0F0
:100350008C918093030185E080930401882780932A
:100360000501ACE3BFE0E2EEF9E0A190BB24E9EDCA
:10037000F9E0EA0DFB1D0E9488240E947D19A2EE7F
:10038000B9E08C918F5F8C9310F40C949F0182E004
:10039000809303018EE180930401882780930501F7
:1003A000EAEBFCE40E945A230E94851984E08093C2
:1003B00003018EE180930401882780930501E2EC1C
:1003C000FCE40E945A230E94851986E08093030171
:1003D0008EE180930401882780930501EAECFCE418
:1003E0000E945A230E9485190E94FB010E94FB1A59
:1003F0000E94080208950027A6E3B0E08C9184FBD8
:100400000EF401E040E0041711F00C94FB01089594
:1004100080E693E1A1E0B1E08D939C9382E390E0CC
:10042000909349008093480082E390E00E94A619CF
:1004300082E08093030188E08093040181E080934F
:100440000501E2EDFCE40E945A230E94851985E033
:100450008093030188E18093040181E0809305018A
:10046000E4EBFCE40E945A230E94851988EC90E09A
:10047000909349008093480082E390E00E94A6197F
:100480000027A6E3B0E08C9184FB0EF401E041E08C
:10049000041711F00C940E0208950E94FB1A82EECC
:1004A0009FE0A1E0B1E08D939C9388E080930301ED
:1004B00081E08093040181E080930501EAEDFCE492
:1004C0000E945A230E948519A2EBB9E08C919927CA
:1004D000909349008093480080E693E1A1E0B1E069
:1004E0008D939C9382E08093030181E080930401CB
:1004F0008827809305010E94F31BACE0B1E00E94C5
:100500007F1985E08093030181E0809304018827AF
:10051000809305010E94F31BA5E1B1E00E947F19C1
:10052000409106010091EF09041711F40C94B602F2
:100530000E94F31BACE0B1E00E946B1903E00E9443
:1005400071190E94F31BA5E1B1E00E946B190E9492
:100550007619C59A81E090E00E94A619C59881E0BD
:1005600090E00E94A61980E08093B2098091060174
:100570008093EF09A2EBB9E08C918C5F8C930027FC
:10058000A6E3B0E08C9184FB0EF401E040E0041798
:1005900011F00C94CC0208950027A1E2B0E08C91F8
:1005A00084FB0EF401E040E0041781E009F080E0F4
:1005B0008F930027A1E2B0E08C9185FB0EF401E05F
:1005C00040E0041781E009F080E09F91892B8F9330
:1005D0000027A1E2B0E08C9182FB0EF401E040E044
:1005E000041781E009F080E09F91892B8F93002709
:1005F000A1E2B0E08C9183FB0EF401E040E004172F
:1006000081E009F080E09F91892B882311F40C94FC
:100610000D0382E390E00E94A6190027A1E2B0E05A
:100620008C9183FB0EF401E040E0041711F00C9470
:100630001E03809109018150809309010027A1E2E6
:10064000B0E08C9182FB0EF401E040E0041711F061
:100650000C942F03A9E0B1E08C918F5F8C9300275D
:10066000A1E2B0E08C9184FB0EF401E040E00417BD
:1006700011F00C9440038091070181508093070191
:100680000027A1E2B0E08C9185FB0EF401E040E090
:10069000041711F00C945103A7E0B1E08C918F5F27
:1006A0008C93009107010F3F11F00C945F038BE3D3
:1006B0008093070180910801815080930801009187
:1006C00007010C3311F00C946D0380E08093070157
:1006D000A8E0B1E08C918F5F8C93009108010F3FEF
:1006E00011F00C94760387E18093080100910801D2
:1006F000083111F00C947F0380E080930801009191
:100700000901003011F00C948D038FE180930901F1
:1007100080910A01815080930A0100910901003201
:1007200011F00C949B0381E080930901AAE0B1E0F1
:100730008C918F5F8C9300910A01003011F00C9422
:10074000A4038CE080930A0100910A010D3011F09E
:100750000C94AD0381E080930A010C946402089527
:100760000E94FB1A80E693E1A1E0B1E08D939C9397
:1007700082E08093030181E08093040188278093C5
:100780000501ECEEFCE40E945A230E948519E1E089
:10079000F0E00E948C190E94FB1A0E940802379A0E
:1007A0000E94FB1A82EE9FE0A1E0B1E08D939C9342
:1007B00080E08093F20907B1007EA2EFB9E08C914E
:1007C00090E0890F082707B90E942920A0EFB9E01F
:1007D0008D939C93A2EFB9E08C918F5F8C93A2EFE5
:1007E000B9E08C918093030181E080930401882714
:1007F00080930501E6EFFCE40E945A230E948519CC
:10080000A2EFB9E08C918093030181E08093040111
:10081000882780930501ACE3BFE0E0EFF9E00E9498
:100820002F240E947D190091F209073018F011F071
:100830000C941C040C941F0480E08093F2090027A0
:10084000A6E3B0E08C9184FB0EF401E040E00417D5
:1008500011F00C9430040E94FB1A0E9408020895C3
:1008600081E08093030188E28093040188278093CC
:100870000501ECEFFCE40E945A230E94851982E0F6
:100880008093030188E28093040188278093050107
:10089000E0E0FDE40E945A230E94851983E08093E2
:1008A000030188E280930401882780930501E6E034
:1008B000FDE40E945A230E94851984E0809303017D
:1008C00088E280930401882780930501EAE0FDE433
:1008D0000E945A230E94851985E08093030188E2D3
:1008E00080930401882780930501E0E1FDE40E94E4
:1008F0005A230E94851986E08093030188E2809341
:100900000401882780930501E6E1FDE40E945A2353
:100910000E94851987E08093030188E28093040197
:10092000882780930501ECE1FDE40E945A230E9490
:10093000851988E08093030188E280930401882769
:1009400080930501E2E2FDE40E945A230E9485198A
:100950000C94DB0308950E94FB1A82EE9FE0A1E055
:10096000B1E08D939C9388E08093030181E08093B4
:10097000040181E080930501ECE2FDE40E945A232A
:100980000E9485198FEF90E0909349008093480072
:10099000A6E0BAE0E4E0FCE40E945A230E94F821B9
:1009A000A2E0BAE0E8E0FCE40E945A230E94F821A9
:1009B00007B1007E026007B90E942920A7EFB9E0C5
:1009C0008D939C93E2E0FAE00E947520E7EFF9E056
:1009D000D190E080FF2400270E9494200E942D21C6
:1009E000EDE0F0E0A3EFB9E00E94A924ECE0FCE424
:1009F0000E945A230E94CE21E3EFF9E00E9470206A
:100A00000E945E21EDE0F0E0A3EFB9E00E94A9248E
:100A1000E6E0FAE00E947520E3EFF9E00E94702022
:100A20000E946D21EDE0F0E0A3EFB9E00E94A9245F
:100A3000E3EFF9E00E947020E0E1FCE40E945A2319
:100A40000E94CE210E94D72118F011F00C942A05A3
:100A50000C944A06ACE3BFE0AF93BF93E3EFF9E039
:100A60000E9470200E94BB1911E001E0BF91AF917C
:100A70000E94D923ECE3FFE0A9EFB9E00E94A4248F
:100A8000E3EFF9E00E947020E4E1FCE40E945A23C5
:100A90000E94CE210E94D72181E008F480E08F934C
:100AA000E3EFF9E00E947020E8E1FCE40E945A23A1
:100AB0000E94CE210E94D72181E010F009F080E051
:100AC0009F918923882311F40C946E05E9EFF9E0D6
:100AD000A9EFB9E00E94A4240C943E06E3EFF9E0EC
:100AE0000E947020ECE1FCE40E945A230E94CE2177
:100AF0000E94D72181E008F480E08F93E3EFF9E0D2
:100B00000E947020E0E2FCE40E945A230E94CE2161
:100B10000E94D72181E010F009F080E09F918923A5
:100B2000882311F40C94B4058AE00E94B519E9EF0A
:100B3000F9E0A881B9810E94A424A9EFB9E0EEE30D
:100B4000FDE40E945A230E942320E881F981A9EF45
:100B5000B9E00E9462190E94A4248AE0481A8827FA
:100B6000580A22960C943E06E3EFF9E00E947020AA
:100B7000E4E0FCE40E945A230E94CE210E94D72187
:100B800081E008F480E08F93E3EFF9E00E947020A9
:100B9000E4E2FCE40E945A230E94CE210E94D72165
:100BA00081E010F009F080E09F918923882311F4FF
:100BB0000C94FA058AE00E94B519E9EFF9E0A881E2
:100BC000B9810E94A424A9EFB9E0E0E4FDE40E9409
:100BD0005A230E942320E881F981A9EFB9E00E94FD
:100BE00062190E94A4248AE0481A8827580A22968B
:100BF0000C943E06E3EFF9E00E947020E8E2FCE48A
:100C00000E945A230E94CE210E94D72181E008F43D
:100C100080E08F93E3EFF9E00E947020ECE2FCE4C7
:100C20000E945A230E94CE210E94D72181E010F019
:100C300009F080E09F918923882311F40C943E06EB
:100C40008AE00E94B519E9EFF9E0A881B9810E9414
:100C5000A424A9EFB9E0E4E4FDE40E945A230E9431
:100C60002320E881F981A9EFB9E00E9462190E946E
:100C7000A4248AE0481A8827580A2296A9EFB9E0E6
:100C80000E946219E6E4FDE40E945A230E94232098
:100C90000C945206A9EFB9E0EAE4FDE40E945A235D
:100CA0000E94232080E693E1A1E0B1E08D939C9324
:100CB00081E08093030181E0809304018827809381
:100CC0000501A9EFB9E00E947F19E3EFF9E00E9466
:100CD0007020E0E1FCE40E945A230E94CE210E9491
:100CE000D72118F011F00C9477060C946508E8E20F
:100CF000FCE40E945A230E94CE21E3EFF9E00E9417
:100D000070200E94D720EDE0F0E0A6E1BAE00E945A
:100D1000A924E6E1FAE00E947520E8E2FCE40E94E2
:100D20005A230E94C5210E94E125EDE0F0E0A6E1F2
:100D3000BAE00E94A924E6E1FAE00E947020E0E314
:100D4000FCE40E945A230E94CE210E94D72110F079
:100D50000C94C606AAE1BAE0E4E5FDE40E945A2339
:100D60000E942320E4E3FCE40E945A230E94CE2147
:100D7000E6E1FAE00E9470200E942D21EDE0F0E013
:100D8000A6E1BAE00E94A9240C94A307E6E1FAE0E8
:100D90000E947020E0E3FCE40E945A230E94CE21CE
:100DA0000E94D72181E008F480E08F93E6E1FAE029
:100DB0000E947020E8E3FCE40E945A230E94CE21A6
:100DC0000E94D72181E010F009F080E09F918923F3
:100DD000882311F40C940807AAE1BAE0E8E5FDE4E1
:100DE0000E945A230E942320ECE3FCE40E945A2331
:100DF0000E94CE21E6E1FAE00E9470200E942D219F
:100E0000EDE0F0E0A6E1BAE00E94A9240C94A3076B
:100E1000E6E1FAE00E947020E0E4FCE40E945A233C
:100E20000E94CE210E94D72181E008F480E08F93B8
:100E3000E6E1FAE00E947020E4E4FCE40E945A2318
:100E40000E94CE210E94D72181E010F009F080E0BD
:100E50009F918923882311F40C943807AAE1BAE002
:100E6000ECE5FDE40E945A230E9423200C94A30782
:100E7000E6E1FAE00E947020ECE3FCE40E945A23D1
:100E80000E94CE210E94D72181E008F480E08F9358
:100E9000E6E1FAE00E947020E4E3FCE40E945A23B9
:100EA0000E94CE210E94D72181E010F009F080E05D
:100EB0009F918923882311F40C947A07AAE1BAE060
:100EC000E0E6FDE40E945A230E942320ECE3FCE4C8
:100ED0000E945A230E94CE21E6E1FAE00E9470208F
:100EE0000E94D720EDE0F0E0A6E1BAE00E94A9243C
:100EF0000C94A307E6E1FAE00E947020E4E3FCE42E
:100F00000E945A230E94CE210E94D72110F40C94F3
:100F1000A307AAE1BAE0E4E6FDE40E945A230E9496
:100F20002320E4E3FCE40E945A230E94CE21E6E160
:100F3000FAE00E9470200E94D720EDE0F0E0A6E1E8
:100F4000BAE00E94A924ACE3BFE0AF93BF93E6E10F
:100F5000FAE00E9470200E94BB1911E001E0BF91ED
:100F6000AF910E94D923ECE3FFE0A9EFB9E00E9422
:100F7000A424E6E1FAE00E947020E8E4FCE40E9488
:100F80005A230E94CE210E94D72118F011F00C9410
:100F9000E9078AE00E94B519E9EFF9E0A881B98173
:100FA0000E94A424A9EFB9E0E8E6FDE40E945A23D8
:100FB0000E942320E881F981A9EFB9E00E9462191B
:100FC0000E94A4248AE0481A8827580A22960C9482
:100FD0005B08E6E1FAE00E947020E8E2FCE40E948F
:100FE0005A230E94CE210E94D72181E008F480E09C
:100FF0008F93E6E1FAE00E947020ECE4FCE40E94AA
:101000005A230E94CE210E94D72181E010F009F0DE
:1010100080E09F918923882311F40C942F088AE0A3
:101020000E94B519E9EFF9E0A881B9810E94A424D2
:10103000A9EFB9E0EEE3FDE40E945A230E942320C9
:10104000E881F981A9EFB9E00E9462190E94A42405
:101050008AE0481A8827580A22960C945B08E6E131
:10106000FAE00E947020E0E5FCE40E945A230E940E
:10107000CE210E94D72181E008F480E08F93E6E141
:10108000FAE00E947020E4E4FCE40E945A230E94EB
:10109000CE210E94D72181E010F009F080E09F91DD
:1010A0008923882311F40C945B08E9EFF9E0A9EF98
:1010B000B9E00E94A424EAE1FAE0A9EFB9E00E94B5
:1010C00062190E94A4240C946D08A9EFB9E0ECE623
:1010D000FDE40E945A230E94232084E080930301B0
:1010E00081E080930401882780930501A9EFB9E08E
:1010F0000E947F19E4E5FCE40E945A230E94CE215D
:10110000E3EFF9E00E9470200E945E21EDE0F0E044
:10111000AAE0BAE00E94A924E8E5FCE40E945A2370
:101120000E94CE21EAE0FAE00E9470200E942D2168
:10113000EDE0F0E0AAE0BAE00E94A924ECE5FCE4CE
:101140000E945A230E94CE21EAE0FAE00E94702019
:101150000E94D720EDE0F0E0AAE0BAE00E94A924C6
:10116000E8E5FCE40E945A230E94CE21EAE0FAE07E
:101170000E9470200E946D21EDE0F0E0AAE0BAE04C
:101180000E94A924EAE0FAE00E947020E4E0FCE476
:101190000E945A230E94CE210E94D72110F00C9465
:1011A000D908AAE0BAE0E4E0FCE40E945A230E94D5
:1011B000F821EAE0FAE00E947020E8E5FCE40E94F1
:1011C0005A230E94CE210E94D72118F011F00C94CE
:1011D000EB080C94F308AAE0BAE0E8E5FCE40E940E
:1011E0005A230E94F821EAE0FAE00E94F925EDE096
:1011F000F0E0AEE0BAE00E94A924EEE0FAE00E943E
:101200003220A2E1BAE0DD92EC92A4E1BAE04D9185
:101210005C91A2E1BAE00D911C910417150710F042
:101220000C94380980E18093E2090091E2090631CB
:1012300018F011F00C943809A2E1BAE08C918A936D
:10124000A2EEB9E08C918A93A4E1BAE08C918A93E2
:10125000A2EEB9E08C918A9380E08A930E94941B5D
:10126000A2EEB9E08C918F5F8C9310F40C94150969
:1012700080E18093E2090091E209063118F011F053
:101280000C945C0980E08A93A2EEB9E08C918A9379
:10129000A2E1BAE08C918A93A2EEB9E08C918A9394
:1012A00081E08A930E94941BA2EEB9E08C918F5F3B
:1012B0008C9310F40C943B09A2E1BAE08D919C91BF
:1012C000A4E1BAE08D939C9382EE9FE0A1E0B1E0AF
:1012D0008D939C93ACE3BFE0AF93BF93E2E0FAE061
:1012E0000E9470200E94BB1911E003E0BF91AF91F2
:1012F0000E94D923ECE3FFE0A9EFB9E00E94A42407
:1013000087E0809303018AE080930401882780931B
:101310000501A9EFB9E00E947F19ACE3BFE0AF93EC
:10132000BF93E6E0FAE00E9470200E94BB1911E032
:1013300003E0BF91AF910E94D923ECE3FFE0A9EF56
:10134000B9E00E94A42487E08093030186E480939F
:101350000401882780930501A9EFB9E00E947F1955
:101360000027A6E3B0E08C9184FB0EF401E040E09E
:10137000041711F00C94C1090E94FB1A0E94080284
:1013800008950027A1E2B0E08C9184FB0EF401E007
:1013900040E0041781E009F080E08F930027A1E28C
:1013A000B0E08C9185FB0EF401E040E0041781E091
:1013B00009F080E09F91892B8F930027A1E2B0E094
:1013C0008C9182FB0EF401E040E0041781E009F00B
:1013D00080E09F91892B8F930027A1E2B0E08C9150
:1013E00083FB0EF401E040E0041781E009F080E0A7
:1013F0009F91892B882311F40C94020A82E390E0D8
:101400000E94A6190027A1E2B0E08C9183FB0EF4A4
:1014100001E040E0041711F00C94200AE0E3FCE442
:101420000E945A230E94CE21E2E0FAE00E9470203E
:101430000E945E21EDE0F0E0A2E0BAE00E94A92463
:101440000027A1E2B0E08C9182FB0EF401E040E0C5
:10145000041711F00C943E0AE0E3FCE40E945A23C6
:101460000E94CE21E2E0FAE00E9470200E946D21ED
:10147000EDE0F0E0A2E0BAE00E94A9240027A1E29A
:10148000B0E08C9184FB0EF401E040E0041711F011
:101490000C945C0AE0E6FCE40E945A230E94CE21F0
:1014A000E6E0FAE00E9470200E945E21EDE0F0E0AC
:1014B000A6E0BAE00E94A9240027A1E2B0E08C9146
:1014C00085FB0EF401E040E0041711F00C947A0A59
:1014D000E0E6FCE40E945A230E94CE21E6E0FAE016
:1014E0000E9470200E946D21EDE0F0E0A6E0BAE0DD
:1014F0000E94A9240C94D80408950E94FB1A82EE3D
:101500009FE0A1E0B1E08D939C930027A3E2B0E0BF
:101510008C9187FB0EF401E041E0041711F00C946C
:10152000A20A87E08093030181E08093040181E0B7
:1015300080930501E6E7FDE40E945A230E94851985
:101540000C94B10A87E08093030181E08093040149
:1015500081E080930501E8E8FDE40E945A230E949F
:1015600085198FEF90E09093490080934800A2E0A6
:10157000BAE0E4E6FCE40E945A230E94F821A6E0C7
:10158000BAE0E8E6FCE40E945A230E94F82107B181
:10159000007E056007B90E942920A7EFB9E08D936E
:1015A0009C93E2E0FAE00E947520E7EFF9E0D19029
:1015B000E080FF2400270E9494200E942D21EDE06E
:1015C000F0E0A3EFB9E00E94A924ACE3BFE0AF9341
:1015D000BF93E3EFF9E00E9470200E94BB1911E075
:1015E00002E0BF91AF910E94D923ECE3FFE0A9EFA5
:1015F000B9E00E94A424E3EFF9E00E947020E4E047
:10160000FCE40E945A230E94CE210E94D72181E04F
:1016100008F480E08F93E3EFF9E00E947020E4E2A9
:10162000FCE40E945A230E94CE210E94D72181E02F
:1016300010F009F080E09F918923882311F40C9425
:10164000410B8AE00E94B519E9EFF9E0A881B98160
:101650000E94A424A9EFB9E0E8E6FDE40E945A2321
:101660000E942320E881F981A9EFB9E00E94621964
:101670000E94A4248AE0481A8827580A22960C94CB
:10168000850BE3EFF9E00E947020E8E2FCE40E94A1
:101690005A230E94CE210E94D72181E008F480E0E5
:1016A0008F93E3EFF9E00E947020ECE2FCE40E94EB
:1016B0005A230E94CE210E94D72181E010F009F028
:1016C00080E09F918923882311F40C94850B8AE094
:1016D0000E94B519E9EFF9E0A881B9810E94A4241C
:1016E000A9EFB9E0EEE3FDE40E945A230E94232013
:1016F000E881F981A9EFB9E00E9462190E94A4244F
:101700008AE0481A8827580A229680E693E1A1E0E9
:10171000B1E08D939C93A9EFB9E00E946219EAE9C8
:10172000FDE40E945A230E94232081E0809303015C
:1017300081E080930401882780930501A9EFB9E037
:101740000E947F19E3EFF9E00E947020ECE6FCE4D0
:101750000E945A230E94CE210E94D72110F00C949F
:10176000B20B1F9A07B1007E076007B90E942920BB
:10177000A7EFB9E08D939C93E2E0FAE00E94752018
:10178000E7EFF9E0D190E080FF2400270E94942049
:101790000E942D21EDE0F0E0A3EFB9E00E94A92422
:1017A000E3EFF9E0A3EFB9E00E94A924E6E0FAE054
:1017B0000E947520E3EFF9E00E9470200E946D21E5
:1017C000EDE0F0E0A3EFB9E00E94A924ACE3BFE0B4
:1017D000AF93BF93E3EFF9E00E9470200E94BB1922
:1017E00011E002E0BF91AF910E94D923ECE3FFE04A
:1017F000A9EFB9E00E94A424E3EFF9E00E94702071
:10180000E4E0FCE40E945A230E94CE210E94D721EA
:1018100081E008F480E08F93E3EFF9E00E9470200C
:10182000E8E4FCE40E945A230E94CE210E94D721C2
:1018300081E010F009F080E09F918923882311F462
:101840000C94420C8AE00E94B519E9EFF9E0A881F6
:10185000B9810E94A424A9EFB9E0E8E6FDE40E9462
:101860005A230E942320E881F981A9EFB9E00E9460
:1018700062190E94A4248AE0481A8827580A2296EE
:101880000C94860CE3EFF9E00E947020E8E2FCE49F
:101890000E945A230E94CE210E94D72181E008F4A1
:1018A00080E08F93E3EFF9E00E947020ECE2FCE42B
:1018B0000E945A230E94CE210E94D72181E010F07D
:1018C00009F080E09F918923882311F40C94860C01
:1018D0008AE00E94B519E9EFF9E0A881B9810E9478
:1018E000A424A9EFB9E0EEE3FDE40E945A230E948C
:1018F0002320E881F981A9EFB9E00E9462190E94D2
:10190000A4248AE0481A8827580A229680E693E1A0
:10191000A1E0B1E08D939C93A9EFB9E00E94621918
:10192000EAE9FDE40E945A230E94232084E0809388
:10193000030181E080930401882780930501A9EFCA
:10194000B9E00E947F1982EE9FE0A1E0B1E08D93A3
:101950009C93E3EFF9E00E947020E0E7FCE40E9432
:101960005A230E94CE210E94D72118F011F00C9426
:10197000BB0C0C94CC0C88E08093030181E0809335
:10198000040181E080930501ECE9FDE40E945A2303
:101990000E9485190C94DB0C88E08093030181E0A0
:1019A0008093040181E080930501EEEAFDE40E944A
:1019B0005A230E948519E3EFF9E00E947020E4E7C2
:1019C000FCE40E945A230E94CE210E94D72118F0E5
:1019D00011F00C94ED0C0C942B0DE1E0F0E00E9462
:1019E0008C190E94FB1A80E693E1A1E0B1E08D938F
:1019F0009C9382E08093030181E080930401882717
:101A000080930501E0ECFDE40E945A230E948519B1
:101A100084E08093030188E0809304018827809309
:101A20000501E8ECFDE40E945A230E94851986E036
:101A30008093030181E0809304018827809305014E
:101A4000E0EDFDE40E945A230E948519E3E0F0E0F6
:101A50000E948C191F98E3EFF9E00E947020E8E7DC
:101A6000FCE40E945A230E94CE210E94D72110F04C
:101A70000C94780DE1E0F0E00E948C190E94FB1AB2
:101A800080E693E1A1E0B1E08D939C9382E08093A6
:101A9000030188E080930401882780930501E8ED25
:101AA000FDE40E945A230E94851984E0809303017B
:101AB00081E080930401882780930501E0EEFDE436
:101AC0000E945A230E94851986E08093030181E0D9
:101AD00080930401882780930501E0EDFDE40E94D6
:101AE0005A230E948519E3E0F0E00E948C191F98A8
:101AF0000027A6E3B0E08C9184FB0EF401E040E007
:101B0000041711F00C94890D0E94FB1A0E94080220
:101B100008950C94C70A0895979A8AE090E00E946D
:101B2000A6199798089580E08093D1098D9A8E9A8E
:101B30009698A1EDB9E0119698E08E91983018F43E
:101B4000392F992702C038E09850881F959808F4DB
:101B5000959A00000000969A0000000096980000F8
:101B600000003A9591F7992341F782E08093D109DB
:101B70008D9A8E9A9698A1EDB9E0119698E08E9183
:101B8000983018F4392F992702C038E09850881FF0
:101B9000959808F4959A00000000969A00000000BD
:101BA0009698000000003A9591F7992341F780E05C
:101BB0008093D1098D9A8E9A9698A1EDB9E01196ED
:101BC00098E08E91983018F4392F992702C038E0A8
:101BD0009850881F959808F4959A00000000969AEE
:101BE000000000009698000000003A9591F79923B4
:101BF00041F780E08093D1098D9A8E9A9698A1ED55
:101C0000B9E0119698E08E91983018F4392F992701
:101C100002C038E09850881F959808F4959A000003
:101C20000000969A000000009698000000003A9587
:101C300091F7992341F780E08093D1098D9A8E9A8C
:101C40009698A1EDB9E0119698E08E91983018F42D
:101C5000392F992702C038E09850881F959808F4CA
:101C6000959A00000000969A0000000096980000E7
:101C700000003A9591F7992341F781E08093D109CB
:101C80008D9A8E9A9698A1EDB9E0119698E08E9172
:101C9000983018F4392F992702C038E09850881FDF
:101CA000959808F4959A00000000969A00000000AC
:101CB0009698000000003A9591F7992341F780E04B
:101CC0008093D1098D9A8E9A9698A1EDB9E01196DC
:101CD00098E08E91983018F4392F992702C038E097
:101CE0009850881F959808F4959A00000000969ADD
:101CF000000000009698000000003A9591F79923A3
:101D000041F780E08093D1098D9A8E9A9698A1ED43
:101D1000B9E0119698E08E91983018F4392F9927F0
:101D200002C038E09850881F959808F4959A0000F2
:101D30000000969A000000009698000000003A9576
:101D400091F7992341F78CE28093D1098D9A8E9A6D
:101D50009698A1EDB9E0119698E08E91983018F41C
:101D6000392F992702C038E09850881F959808F4B9
:101D7000959A00000000969A0000000096980000D6
:101D800000003A9591F7992341F782E08093D109B9
:101D90008D9A8E9A9698A1EDB9E0119698E08E9161
:101DA000983018F4392F992702C038E09850881FCE
:101DB000959808F4959A00000000969A000000009B
:101DC0009698000000003A9591F7992341F78FEF1C
:101DD0009FE3A7EBB9E08D939C938D9A8E9A96988A
:101DE000A7EBB9E0129690E18E91983018F4392F54
:101DF000992702C038E09850881F959808F4959A62
:101E000000000000969A0000000096980000000074
:101E10003A9591F7992341F7949A0000000094981D
:101E20000895A6EDB9E0E9EBF9E00E948D1FA881C5
:101E3000B981E9ECF9E00E948D1FA9ECB9E0BA93F1
:101E4000AA93ECE7FCE40E945A23A1ECB9E00E94BB
:101E50004D1EE9ECF9E00E94461D2296A9ECB9E07E
:101E6000BA93AA93A9EBB9E0E9ECF9E00E94A51DA9
:101E70002296E9ECF9E0A9ECB9E00E941B1EE9EC1E
:101E8000F9E0A3EBB9E00E94AB1F0895A881B981E6
:101E90000D911C910F3F5FE3150710F40C94560F42
:101EA0008FEF9FE3A881B9818D939C9382E080930B
:101EB000D1098D9A8E9A9698A1EDB9E0119698E085
:101EC0008E91983018F4392F992702C038E0985035
:101ED000881F959808F4959A00000000969A0000D3
:101EE00000009698000000003A9591F7992341F779
:101EF0008D9A8E9A9698A881B981129690E18E91CA
:101F0000983018F4392F992702C038E09850881F6C
:101F1000959808F4959A00000000969A0000000039
:101F20009698000000003A9591F7992341F7949A0A
:101F3000000000009498089584E08093D1098D9A60
:101F40008E9A9698A1EDB9E0119698E08E9198300E
:101F500018F4392F992702C038E09850881F9598B7
:101F600008F4959A00000000969A000000009698E8
:101F7000000000003A9591F7992341F78D9A8E9AC7
:101F80009698A881B981149690E28E91983018F4B1
:101F9000392F992702C038E09850881F959808F487
:101FA000959A00000000969A0000000096980000A4
:101FB00000003A9591F7992341F7949A00000000A8
:101FC0009498089501080800000000000000000037
:101FD0000000065F06000000000703000703000082
:101FE00000247E247E24000000242B6A12000000BE
:101FF0000063130864630000003649562050000057
:10200000000007030000000000003E410000000047
:102010000000413E0000000000083E1C3E08000099
:102020000008083E080800000000E0600000000012
:1020300000080808080800000000606000000000B8
:102040000020100804020000003E5149453E0000F7
:102050000000427F400000000062514949460000F4
:102060000022494949360000001814127F10000070
:10207000002F494949310000003C4A4949300000DD
:102080000001710905030000003649494936000086
:1020900000064949291E000000006C6C0000000089
:1020A0000000EC6C00000000000814224100000059
:1020B00000242424242400000000412214080000ED
:1020C0000002015909060000003E415D551E000056
:1020D000007E1111117E0000007F49494936000041
:1020E000003E414141220000007F4141413E00004D
:1020F000007F494949410000007F090909010000AA
:10210000003E4149497A0000007F0808087F00002E
:102110000000417F4100000000304040403F00008F
:10212000007F081422410000007F40404040000032
:10213000007F0204027F0000007F0204087F00008D
:10214000003E4141413E0000007F090909060000B0
:10215000003E4151215E0000007F09091966000020
:1021600000264949493200000001017F01010000B9
:10217000003F4040403F0000001F2040201F000063
:10218000003F403C403F000000631408146300001F
:10219000000708700807000000714945430000006F
:1021A00000007F41410000000002040810200000F0
:1021B000000041417F000000000402010204000011
:1021C0008080808080808080000003070000000005
:1021D0000020545454780000007F444444380000E8
:1021E000003844444428000000384444447F000040
:1021F000003854545408000000087E09090000000B
:102200000018A4A4A47C0000007F0404780000004F
:102210000000007D40000000004080847D00000040
:10222000007F1028440000000000007F40000000F4
:10223000007C041804780000007C0404780000008E
:10224000003844444438000000FC44444438000052
:102250000038444444FC0000004478440408000072
:10226000000854545420000000043E4424000000A0
:10227000003C40207C000000001C2040201C00008E
:10228000003C6030603C0000006C10106C000000EE
:10229000009CA0603C000000006454544C0000000E
:1022A00000083E41410000000000007700000000EF
:1022B000000041413E080000000201020100000050
:1022C000003C2623263C0000001EA1E12112000054
:1022D000003D40207D0000000038545455090000A6
:1022E00000205555557800000020555455780000C1
:1022F00000205555547800000020575557780000AD
:10230000001CA2E2221400000038555555080000B8
:102310000038555455080000003855555408000041
:102320000000017C41000000000002794200000032
:102330000000017C4000000000702924297000008A
:1023400000782F252F780000007C5454554500005C
:102350000034547C54580000007E097F4949000035
:102360000038454539000000003845443900000078
:102370000039454438000000003C41217D00000048
:10238000003D41207C000000009CA1603D00000059
:10239000003D42423D000000003C41403D00000045
:1023A000001824662400000000483E4949620000ED
:1023B00000292A7C2A290000007F091678100000D5
:1023C0000040887E09020000002054555578000026
:1023D0000000007D41000000003844453900000045
:1023E000003C40217D000000007A090A71000000D5
:1023F000007A11227900000000085555555E000052
:10240000004E51514E0000000030484D4020000069
:10241000003C04040404000004040404041C000040
:102420000017084C6A500000001708342A78000092
:102430000000307D30000000000814000814000087
:102440000014080014080000441144114411000055
:10245000AA55AA55AA550000BBEEBBEEBBEE000084
:10246000000000FF00000000080808FF0000000056
:102470000A0A0AFF0000000008FF00FF0000000039
:1024800008F808F8000000000A0A0AFE0000000030
:102490000AFB00FF0000000000FF00FF000000003A
:1024A0000AFA02FE000000000A0B080F00000000FC
:1024B000080F080F000000000A0A0A0F00000000C1
:1024C000080808F8000000000000000F08080000DD
:1024D0000808080F08080000080808F808080000A5
:1024E000000000FF080800000808080808080000AD
:1024F000080808FF08080000000000FF0A0A0000A2
:1025000000FF00FF08080000000F080B0A0A000087
:1025100000FE02FA0A0A00000A0B080B0A0A000071
:102520000AFA02FA0A0A000000FF00FB0A0A000089
:102530000A0A0A0A0A0A00000AFB00FB0A0A00004B
:102540000A0A0A0B0A0A0000080F080F0808000010
:102550000A0A0AFA0A0A000008F808F8080800003F
:10256000000F080F080800000000000F0A0A000012
:10257000000000FE0A0A000000F808F80808000041
:1025800008FF00FF080800000A0A0AFB0A0A000008
:102590000808080F00000000000000F8080800000C
:1025A000FFFFFFFFFFFF0000F0F0F0F0F0F0000091
:1025B000FFFFFF0000000000000000FFFFFF000021
:1025C0000F0F0F0F0F0F0000001824241824000015
:1025D00000FE4A4A34000000007F010103000000B1
:1025E00000027E027E020000006355496300000085
:1025F000001824241C04000000FC20201C00000003
:102600000008047804000000000855775508000011
:10261000003E49493E000000004C7202724C00002E
:10262000002255593000000000182418241800001A
:102630000018247E24180000001C2A2A2A0000000A
:10264000003C02023C000000002A2A2A2A00000066
:102650000000242E2400000000514A4A44000000DB
:1026600000444A4A51000000000000FC020400003F
:102670000020403F000000000008082A0808000071
:1026800000241224120000000006090906000000C0
:102690000000181800000000000008000000000002
:1026A0000030403E0202000000010E010E0000005A
:1026B00000090D0A00000000003C3C3C3C0000000A
:1026C00002102000000000000000000000000000D8
:1026D00000000000000000000000000000000000FA
:1026E000000000000000000000007CFFFF7C0000F4
:1026F0000000000000000000000000333300000074
:102700000000000000000000003C3C00003C3C00D9
:1027100000000000000000000000000000000000B9
:102720000000000000001090F07E1E90F07E1E1051
:102730000000000000021E1F03021E1F0302000013
:10274000000000000000000078FCCCFFFFCCCC882B
:102750000000000000000000040C0C3F3F0C0F07BD
:10276000000000000000001C1C1C80C0E070381C31
:102770000E0000000000181C0E070301001C1C1CAA
:10278000000000000000000000B8FCC6E23E1C0093
:1027900000000000000000001F3F3121371E1C36E2
:1027A00022000000000000000000273F1F00000082
:1027B0000000000000000000000000000000000019
:1027C00000000000000000F0FCFE07010100000016
:1027D00000000000000000030F1F38202000000050
:1027E000000000000000000000010107FEFCF000F6
:1027F0000000000000000000002020381F0F030030
:1028000000000000000000004C5CF0FCFCF05C4CA0
:10281000000000000000000006070107070107068E
:102820000000000000000000808080F0F0808080C8
:1028300000000000000000000101010F0F01010174
:102840000000000000000000000000000000000088
:102850000000000000000000000000B8F878000050
:102860000000000000000000808080808080808068
:102870000000000000000000010101010101010150
:102880000000000000000000000000000000000048
:102890000000000000000000000000383838000090
:1028A000000000000000000000000080C0E0703860
:1028B0001C0E0600000000181C0E0703010000009B
:1028C00000000000000000F8FE060383C363331E0F
:1028D000FEF80000000000071F1E333130303018B2
:1028E0001F07000000000000000C0C0EFFFF00009E
:1028F0000000000000000000003030303F3F30306A
:10290000300000000000001C1E07030383C3E377B0
:102910003E1C000000000030383C3E373331303080
:10292000303000000000000C0E07C3C3C3C3C3E770
:102930007E3C00000000000C1C3830303030303954
:102940001F0E0000000000C0E070381C0E07FFFFE3
:1029500000000000000000030303030303033F3FE4
:10296000030300000000003F7F636363636363E36E
:10297000C38300000000000C1C3830303030303889
:102980001F0F000000000000C0F0F8DCCEC7C3C37A
:10299000C3800000000000070F1F39303030303096
:1029A000391F0F00000000030303030303C3F33FB9
:1029B0000F030000000000000000303C0F03000087
:1029C00000000000000000BCFEE7C3C3C3E7FEBC7C
:1029D0000000000000000F1F393030303030391F48
:1029E0000F0000000000003C7EE7C3C3C3C3C3E781
:1029F000FEFC00000000000000303030381C0E07E4
:102A00000300000000000000000000707070000073
:102A100000000000000000000000001C1C1C000062
:102A20000000000000000000000000707070000056
:102A300000000000000000000000009CFC7C000082
:102A4000000000000000C0E0F0381C0E070300008A
:102A5000000000000000000103070E1C38300000D9
:102A60000000000000000000606060606060606066
:102A700060000000000000000606060606060606C6
:102A80000600000000000000000003070E1C38F0E4
:102A9000E0C0000000000000000030381C0E0703FA
:102AA000010000000000001C1E070383C3E3773E03
:102AB0001C0000000000000000000037370000008C
:102AC000000000000000F8FE07F3FB1BFBFB07FE05
:102AD000F800000000000F1F183337363737360371
:102AE000010000000000000000E0FC1F1FFCE000EF
:102AF00000000000000000383F0706060606073FFA
:102B000038000000000000FFFFC3C3C3C3E7FEBCE2
:102B1000000000000000003F3F3030303030391FEF
:102B20000F000000000000F0FC0E07030303070E77
:102B30000C000000000000030F1C38303030381C3F
:102B40000C000000000000FFFF03030303070EFC5E
:102B5000F00000000000003F3F30303030381C0FE4
:102B60000300000000000000FFFFC3C3C3C3C3C3D2
:102B700003030000000000003F3F303030303030B1
:102B800030300000000000FFFFC3C3C3C3C3C30352
:102B9000030000000000003F3F00000000000000B4
:102BA0000000000000000000F0FC0E0703C3C3C3D8
:102BB000C7C6000000000000030F1C383030303062
:102BC0003F3F0000000000FFFFC0C0C0C0C0C0FF0A
:102BD000FF0000000000003F3F0000000000003F39
:102BE0003F00000000000000000303FFFF0303009C
:102BF00000000000000000000030303F3F30300097
:102C0000000000000000000000000000000000FFC5
:102C1000FF0000000000000E1E3830303030381F3A
:102C200007000000000000FFFFC0E0F0381C0E07A6
:102C3000030000000000003F3F000103070E1C38A6
:102C400030000000000000FFFF0000000000000056
:102C5000000000000000003F3F30303030303030A6
:102C600030000000000000FFFF1E78E0E0781EFF4B
:102C7000FF0000000000003F3F0000010100003F96
:102C80003F000000000000FFFF0E38F0C00000FF12
:102C9000FF0000000000003F3F00000003071C3F52
:102CA0003F000000000000F0FC0E070303070EFCCD
:102CB000F0000000000000030F1C383030381C0FFB
:102CC00003000000000000FFFF8383838383C7FEAF
:102CD0007C0000000000003F3F01010101010100F4
:102CE00000000000000000F0FC0E070303070EFCCC
:102CF000F0000000000000030F1C3830363E1C3F7F
:102D000033000000000000FFFF8383838383C7FE3E
:102D10007C0000000000003F3F010103070F1D3849
:102D2000300000000000003C7EE7C3C3C3C3C78E71
:102D30000C0000000000000C1C3830303030391F0F
:102D40000F00000000000000030303FFFF03030364
:102D500000000000000000000000003F3F000000F5
:102D600000000000000000FFFF000000000000FF66
:102D7000FF000000000000071F3830303030381FDF
:102D800007000000000000073FF8C00000C0F83F47
:102D9000070000000000000000010F3E3E0F010090
:102DA00000000000000000FFFF000080800000FF26
:102DB000FF0000000000003F3F1C060303061C3F0D
:102DC0003F000000000000030F1C30E0E0301C0F4B
:102DD00003000000000000303C0E030101030E3C24
:102DE00030000000000000030F3CF0C0C0F03C0FBA
:102DF00003000000000000000000003F3F00000052
:102E00000000000000000003030303C3E3331F0FAF
:102E100003000000000000303C3E333130303030E1
:102E2000300000000000000000FFFF030303030068
:102E30000000000000000000003F3F303030300054
:102E400000000000000E1C3870E0C0800000000090
:102E5000000000000000000000000103070E1C1825
:102E60000000000000000003030303FFFF00000058
:102E700000000000000000303030303F3F00000014
:102E800000000000006070381C0E070E1C387060D7
:102E90000000000000000000000000000000000032
:102EA0000000000000000000000000000000000022
:102EB00000000000000000C0C0C0C0C0C0C0C0C052
:102EC000C0C000000000000000003E7E4E00000078
:102ED00000000000000000000000000000000000F2
:102EE000000000000000000040606060606060E082
:102EF000C00000000000001C3E3333333333333F47
:102F00003F000000000000FFFFC060606060E0C0A4
:102F1000800000000000003F3F3030303030381F6C
:102F20000F00000000000080C0E06060606060C0D2
:102F3000800000000000000F1F38303030303018A3
:102F40000800000000000080C0E0606060E0C0FF9A
:102F5000FF0000000000000F1F3830303030303FDD
:102F60003F00000000000080C0E06060606060C062
:102F7000800000000000000F1F3B33333333331356
:102F800001000000000000C0C0FCFEC7C3C3030076
:102F90000000000000000000003F3F0000000000B3
:102FA0000000000000000080C0E06060606060E041
:102FB000E000000000000003C7CECCCCCCCCE67F04
:102FC0003F000000000000FFFFC0606060E0C080C4
:102FD000000000000000003F3F00000000003F3FF5
:102FE0000000000000000000000060ECEC000000A9
:102FF00000000000000000000030303F3F30300093
:1030000000000000000000000000000060ECEC0088
:1030100000000000000000000060E0C0C0FF7F0072
:10302000000000000000000000FFFF0080C0E06022
:103030000000000000000000003F3F03070F1C38A5
:103040003000000000000000000003FFFF0000004F
:1030500000000000000000000030303F3F30300032
:1030600000000000000000E0C0E0E0C0C0E0E0C000
:10307000800000000000003F3F00003F3F00003F95
:103080003F00000000000000E0E060606060E0C021
:1030900080000000000000003F3F00000000003FF3
:1030A0003F00000000000080C0E060606060E0C0A1
:1030B000800000000000000F1F3830303030381F13
:1030C0000F000000000000E0E06060606060E0C0B1
:1030D00080000000000000FFFF0C181818181C0FDB
:1030E0000700000000000080C0E06060606060E0F9
:1030F000E0000000000000070F1C181818180CFF53
:10310000FF00000000000000E0E0C060606060E0E0
:10311000C0000000000000003F3F00000000000071
:103120000000000000000000C0E0606060606040DF
:1031300000000000000000001133333333333F1E22
:1031400000000000000000006060FEFE60606000A3
:10315000000000000000000000001F3F3030303051
:1031600000000000000000E0E0000000000000E0BF
:10317000E00000000000000F1F3830303030183FF2
:103180003F00000000000060E0800000000080E0E0
:10319000600000000000000001071E38381E070113
:1031A00000000000000000E0E00000E0E00000E0BF
:1031B000E0000000000000071F381C0F0F1C381F24
:1031C000070000000000000060E0C0800080C0E058
:1031D000600000000000000030381D0F070F1D3890
:1031E00030000000000000000060E080000080E08F
:1031F0006000000000000000000081E77E1E070163
:1032000000000000000000006060606060E0E060BE
:10321000200000000000000030383C3633313030F0
:1032200030000000000080C0FC7E070303030000A4
:1032300000000000000000011F3F7060606000009F
:10324000000000000000000000FFFF000000000080
:103250000000000000000000003F3F0000000000F0
:10326000000000000000000000030303077EFCC014
:10327000800000000000000000606060703F1F01DF
:103280000000000000000010180C040C1810180CAE
:10329000040000000000000000000000000000002A
:1032A0000000000000000080C0603018183060C0CE
:1032B0008000000000000007070606060606060755
:1032C000070000008F938D918823E9F711978F9164
:1032D0000895ACE3BFE08D91882311F00AD0FBCFB5
:1032E000089580E206D00A95E9F708958DE001D0AF
:1032F0008AE05D9BFECF8CB90895ACE3BFE08D9171
:10330000882311F00FD0FBCF08950E94BB21802DA0
:1033100011F008D0FACF089588EE93E017D03197D6
:10332000D9F708950C940F1B3197F1F70895B99AC6
:10333000BB98C39ABA9A8CE58DB9089508950895FB
:10334000689462F80895E89462F80895EF93FF9303
:10335000EE27E82BE92B31F0EDECFAE03197F1F7AD
:103360000197D1F7FF91EF9108955A924A92480E32
:103370008827581E08958DE207FD8D938F2D881F95
:10338000802F881F8F57082F6894F7F8802F87FFAA
:1033900015C080958395082F80E38D938EE28D93E1
:1033A000802F815228F080E38D9399279C93089574
:1033B00044270A95802F09F198D01FC0805230F021
:1033C0009EE49D9381E48D939D93EFCF4427DF92FC
:1033D000EF92FF920F938FE1801B11F0082F85D0A1
:1033E0008BD09EE29D930F91FF90EF90DF9044274A
:1033F0000395003209F4D7CF2DD03F93EAE8F4E3E8
:103400000E945A2338E12F2D1E2D0D2DFF24EE246E
:10341000DD244427000F111F221FA8F42F923F9292
:103420000E94BB21102C0E94BB21202C0E94BB219A
:10343000302C0E94BB213197410DD21CE31CF01CA3
:103440003F902F9001C0339631963A9519F73F91EE
:1034500007D0ADCFDD0CEE1CFF1C0A95D9F70895FF
:10346000002719E058D08F93802B11F0039501C0ED
:103470008F911A95B9F7802F882309F494CF8F91F3
:10348000805D8D930A95D9F790CF0065CD1D80B2F0
:10349000E60E40597307A0ACB90350D6DC01286B87
:1034A000EE0094357700CA9A3B0065CD1D00B2E668
:1034B0000E0059730700ACB90300D6DC01006BEEB7
:1034C0000000357700009A3B0000CD1D0000E60E9D
:1034D000000073070000B9030000DC010000EE00EB
:1034E0000000770000003B000000F694E794D794BA
:1034F00047950A95D1F7089500270DD08F9303952E
:103500008F2D8E298D29842BC1F78F91805D8D930E
:103510000A95D9F74ACF1F930F93002710E2440F63
:10352000DD1CEE1CFF1C001F802F9AE0890B10F0A1
:10353000082F43951A9599F7802F0F911F910895A1
:10354000442718D0AD98AC9AAA9884E699270E948F
:10355000A6199FEF9ABBAD9A2ED014FCFDCF02D0D6
:103560004FEF08D08FE30FD080EC0DD080E40BD06C
:1035700088EB09C0403420F0AF9AAE9840540895CB
:10358000AE9AAF980895AB9801C0AB9AEF93FF93B2
:10359000EAE0F0E00E949419FF91EF918BBBAC98A8
:1035A000AA9AEF93FF93E2E0F0E00E949419FF9152
:1035B000EF91AA980895AB9804D017FCFCCF08951A
:1035C000AB9A99279ABB9FEF9BBBEF93FF93EAE0DF
:1035D000F0E00E949419FF91EF91AC9AAA9AEF93B0
:1035E000FF93E2E0F0E00E949419FF91EF9119B28D
:1035F000AA989ABB08954427BDDF02D04FEFBADFE7
:1036000000E080E4C0DF88EB800FBDDF10E4882796
:10361000BCDF1A95E1F70395083099F70895EF9309
:10362000FF931BB61F92509103015F9370900401AA
:10363000E0910101F09102010024EE0FFF1F001C38
:103640000BBE0E94BB21202D0E94BB21302D0E9469
:10365000BB21002D0E94BB218052482F0E94AF2425
:10366000E40FF51F27D070920401732F40910401DD
:103670005091030129D00E94BB21802D509105015A
:10368000552309F0809581DF5091040153955093A3
:1036900004017A9559F75091030153955093030112
:1036A0002A9509F75F91509303011F901BBEFF916C
:1036B000EF91089518F42BB623942BBE089518F4B7
:1036C0002BB62A942BBE08954A955A9553DF88EB62
:1036D000850F59DF80E4840F56CF0F921F922F92EF
:1036E0003F920F939F934F93052F48E00E94BB2476
:1036F000082E4F91502F242E352EE8DF61DF60DF3A
:10370000422D532DE3DF802D0E9406220F910023CE
:1037100011F0182A01C01922812D37DF0F913F9037
:103720002F901F900F900895AA24BB24FF24EC81B2
:10373000EA80EE1AFF08FB81298033242F1A330810
:1037400081E0EA14FA043CF42FEF3FEFE094F094A8
:10375000E80EFA1C02C021E033272A143A043CF494
:103760006FEF7FEF20943094280E3A1C02C061E086
:10377000772735D02E143F0414F009F017C0CE2C53
:10378000DF2CCC0CDD1C022C132C000C111C9A819C
:10379000E91761F0E20FA00CB11CAE14BF0424F0D5
:1037A00019F0F60FAC18BD081AD0F1CFC22CD32CEB
:1037B000CC0CDD1C0E2C1F2C000C111C9981F91750
:1037C00011F425960895F60FA00CB11CA214B304B1
:1037D00024F019F0E20FAC18BD0801D0EFCF4E2F46
:1037E0005F2F98817ACFACE0B1E0E9E0F1E00E9490
:1037F000401C33970C941C1CECE0F1E0A9E0B1E014
:103800000E942E1CE5E1F1E0A6E0B1E00E940A1C56
:10381000ADE0BB27868197810E946E230D93838143
:1038200094810E946E230D93808191810E946E236A
:103830000D930895EDE0FF2782810E9463238AE3C0
:103840008D9381810E9463238AE38D9380810E94FE
:10385000632388278C930895ADE0BB2786819781E9
:103860000E946E230D93838194810E946E230D9399
:10387000808191810E946E230D930895EDE0FF27D2
:1038800082810E9463238DE28D9381810E94632354
:103890008DE28D9380810E94632388278D93089504
:1038A000C09846D0072F44D0062F42D0052F40D0D5
:1038B000042F3ED01F932F93112725E0E89435D095
:1038C0000F3F21F411502040D1F768942F911F91A0
:1038D00000230895C09A1AE028D01A95E9F7C098F5
:1038E00000E426D024D023D022D021D005E920D056
:1038F00014E6E0DF013021F01A95D9F791EE79C096
:1039000073C01AE0C09801E413D011D010D00FD0CA
:103910000ED0D0DF49F068D082E390E00E94A61973
:103920001A9581F792EE65C05FC00FEF01C00027C6
:103930000FB9779BFECF0FB1089544275D916D912C
:103940007D91550F661F771F089545D0F6DF01E57D
:10395000A7DF11F093EE4DC0ADDF0E3F11F095EEF5
:1039600048C092E08827E1DF01930197E1F7DDDFAE
:10397000DCDF3AC030D0E1DF08E592DF11F094EEF1
:1039800038C0D3DF0EEFD4DF92E088270191D0DF7B
:103990000197E1F7CADFC9DFC8DF0F71009321018A
:1039A00011272FEF31D0C1DF002329F4115020401F
:1039B000C9F796EE1EC018C00E9497190CD08ADF76
:1039C00008F408959ECF07D085CF05D081E00EC0C2
:1039D00002D098EE13C09927889490931E0190937B
:1039E000200190931F010895C09A9FDF9927889422
:1039F000089504D0C09A99DF0894089590931E0109
:103A0000009320010894089595E29A95F1F708959E
:103A10002DD204D05BC10F0101D05BC100E03DD2CB
:103A200009F008959A01281B390B1AF4D0010F01EF
:103A3000F5CF00272733300708F064C2822F79D1F1
:103A40008DD19BD1372F36270AF4BFD1F001808169
:103A5000A80E8181B81E8281C81E8381D81E8481F0
:103A6000E81E8581F81E86818F708061081F1AF418
:103A7000ACD180E8682705FF02C081E07CD104FD5D
:103A800001C0D6D194C1F2D104D020C10F0101D020
:103A900020C108E102D209F00895480F591F4F5F75
:103AA000534067276F935F934F93E6D12227F0012E
:103AB0004BD193E0110F331F441F551F661F771F13
:103AC000881F9A95B9F7FD01A7E0BB279191A13016
:103AD00011F49F709061992301F1939FA00CB11C88
:103AE000BB1F959FB695C01CD11CBB1F979FB69559
:103AF000E01CF11C0B1F919F200DA11CBB1F949F6C
:103B0000B695B01CC11CBB1F969FB695D01CE11C7E
:103B1000BB1F989FB695F01C011DAA9549F02A2D50
:103B2000AB2CBC2CCD2CDE2CEF2CF02E0027CECFD6
:103B30004F915F916F9104FB16F030D102C04F5F3F
:103B40005F4F35C193D104D0C1C00F0101D0C1C0B6
:103B500004E2A3D109F00895481B590B41505C4F72
:103B600067276F935F934F93F001E3D02FEFFD0131
:103B7000EBD0ADE3BA2FB77019F420952F932FEF48
:103B8000A116B306C406D506E606F706080738F000
:103B9000A11AB30AC40AD50AE60AF70A080B221FBB
:103BA000AA0CBB1CCC1CDD1CEE1CFF1C001FAA9524
:103BB00009F72095AF90BF90CF90DF90EF90FF90E6
:103BC0000F914F915F916F9104FB1EF0E7D0415030
:103BD0005040EDC0E881F981AA81BB810895FADFE8
:103BE0007BD0FD0181D0AC0199273F7711F54F5F64
:103BF00053401AF441D19FEF57C05523D1F44533B8
:103C0000C0F441954C5C9927483030F08081982B66
:103C1000882781934850F8CF7FEF8081442319F0A3
:103C2000770F4A95FBCF672F60956823962B8723E4
:103C300080830895CFDF50D0FD0156D0AC013F778F
:103C4000C9F48E5F934012F417D12EC0992391F4DA
:103C5000863380F487818F938F778783FF93EF93E9
:103C60000AD0EF91FF9187819F919078892B87836C
:103C7000DF01B6CF0895E6EEFFE30E945A2300C0AD
:103C80005D01FF93EF93CBD1EF91FF9106D0F5014A
:103C9000FA93EA93C0DE2296D0C188E007900D9295
:103CA0008A95E1F718970895A082B182C282D382E3
:103CB000E482F582068317830895A080B180C280D4
:103CC000D380E480F580068117810895EC81FD8121
:103CD000EBCFE881F981E8CF88E091919D938A95B7
:103CE000E1F718973897089586819781332797FBD6
:103CF00037F988949F7721F4882311F4326008956E
:103D00002FEE28172FE7290740F42FE028230894E7
:103D100011F43160089534600895807F96958795F9
:103D20009695879596958795969587959894889476
:103D30000895A080B180C280D380E480F5800681A0
:103D40000F700061222708951081318142815381D3
:103D50006481758186818F7080610895883050F00C
:103D60002A2DAB2CBC2CCD2CDE2CEF2CF02E0027DA
:103D70008850F4CF0895689401C0E894882369F0CE
:103D80000595F794E794D794C794B794A79427958B
:103D900016F44F5F5F4F8A95F1CF0895220FAA1C4A
:103DA000BB1CCC1CDD1CEE1CFF1C001F089501D0A9
:103DB00025C0203848F011F4A0FE06C0089412D0A7
:103DC00005FF089581E0D7CF08952095A094B09481
:103DD000C094D094E094F09400950F92002408943D
:103DE000201D0F9050F40F920024A01CB01CC01C8A
:103DF000D01CE01CF01C001D0F9008955523B2F05C
:103E0000352F342B99F03FEF431737E0530778F401
:103E1000440F551F440F551F440F551F440F551F86
:103E20000F7E042B152F67FB17F9089525C02BC0B3
:103E300087E03F2D303230E0030778F40F2DFE2C61
:103E4000ED2CDC2CCB2CBA2CA22E22274850504033
:103E50008A9579F7442755270FC088E004FD05C0EF
:103E60009DDF415050408A95C9F70895EA81FB8152
:103E7000A881B9810F010895AA24BB2465017501A9
:103E8000850198940895F8DF00EF1FE708958FEFFC
:103E9000A82EB82EF3DF1F77089526DF632FAC011D
:103EA000FD0122DF732F00C0372F362B3F7709F437
:103EB000089532FDECCF262F2727372F60FB32F9EC
:103EC00061FB33F93F70EEEEFFE30E945A230023BB
:103ED00011F427FD3C96030FE00F0027F01F869199
:103EE00087FDD5CF86FDCFDF85FDC6DF84FD0AD0F7
:103EF00083FD0AD082FD0AD081FD0BD080FD0BD05E
:103F000098940895F001D9CEFD01D7CE67FB17F93B
:103F1000089577FBFCCF27FBFACFCD90DD90ED9095
:103F2000FD90AA24BB240027112722276627FF2003
:103F300012F406D0606843E254E07ADF5FDFB4CE6B
:103F4000C094D094E094F09481E0C80E8827D81EE5
:103F5000E81EF81E0895C8DE31FD19C032FD17C0F5
:103F600030FD2AC08E5F934092F0992329F580326C
:103F700038F4DFDE81958B5DF1DEE894FEDE0CC067
:103F8000CC24C094DC2CEC2CFC2CF69412C0CC2459
:103F9000DD24EE24FF2410C080E8B81650F031F480
:103FA000BA28B22AB81611F4C0FC03C0CDDFF7FC62
:103FB000E7CF37FF01C0C4DFCD92DD92ED92FD92D5
:103FC0000895B7FE089590E8B91611F4D0FE08954B
:103FD0009FEFD91AE90AF90A09F403950895000038
:103FE00000000000F03F000000000000E03F00087B
:103FF00010001010100008082000000810001080A9
:10400000100008082000004120004141800020806D
:10401000200000204400418044002020800088E0EF
:104020000FB6F8945A924A92E42DF52DA42DB52D91
:10403000480E8827581E0FBE08950FB6F894499071
:1040400059900FBE08950E94BB210D920020D9F710
:104050000895369A3699FECF369A3699FECF84B1B6
:1040600095B108953DD0992711278F2D880F80E8AD
:10407000F82A802F881F08F41FEF41F08F57082F70
:1040800007FD04C0003240F08FEF01C08827982F51
:10409000D82EE82EF82E09C08FE1801B082FF69449
:1040A000E794D79497950A95D1F7112351F09095FD
:1040B000D094E094F09481E0980F8827D81EE81EF1
:1040C000F81E0F2DFE2CED2CD92E0895D094E094DF
:1040D000F09491E0D90E9927E91EF91E10950895E4
:1040E000D190E190F1900191089521913191419108
:1040F00051910895102F90E8FF0C001F0927990F88
:10410000F7941078652F90E8440F551F5927990FA1
:104110004795607800380895FF0C90E89027110FBC
:104120009795F794092F0895102FBD2CDE2CEF2CB6
:10413000F02E11234AF4B094D094E094F0949FEFC1
:10414000B91AD90AE90AF90A0EE1FF2039F4FE2C5E
:10415000ED2CDB2CBB240850C2F75DC032F00A9571
:10416000BB0CDD1CEE1CFF1CF9CF2BDFD5CFDD9285
:10417000ED92FD920C930895502F2D2D3E2D4F2D35
:10418000612F08952DEC3CEC4CEC5DE366270FC0ED
:10419000A7DFF2DFDD24EE2490E8F92E0FE307C05D
:1041A000A4DF05C02227332740E251E466275523C8
:1041B00051F1002381F19EDF71F11627005850580C
:1041C0000894050B18F407FD03C025C007FD23C0A4
:1041D000469537952795F694E794D79422D0FF20FB
:1041E0002AF0DD0CEE1CFF1C015073F09D2D9695FE
:1041F00048F0DD203AF4EE202AF491E0D90E992718
:10420000E91EF91E89CF07C09FE7092FF92A9FEF02
:10421000D92EE92E0895DD24EE24FF24002711274E
:1042200008959F929924AA24BB2488E1D216E3061C
:10423000F40628F0D21AE30AF40A089401C088941C
:10424000991CAA1CBB1CDD0CEE1CFF1C8A9571F787
:10425000D92CEA2CFB2C9F9008954CDFE1F25038CA
:10426000D1F21627005850580894051F12F418F47C
:10427000CBCF08F0D0CF0AD0FF202AF0BB0CDD1C3A
:10428000EE1CFF1C49CF0F5FFBF146CF9F92992494
:10429000AA24BB24992788E1990CAA1CBB1CDD1C0D
:1042A000EE1CFF1C30F4920EA31EB41ED91EE91E94
:1042B000F91E8A9589F79F90089517DF1BDF503804
:1042C00029F090E869270CC00AF045D025CF5FE3BC
:1042D00022273327442701C008DF0CDF5038B1F311
:1042E000003899F3902F951B8BF312F434D0FACF4A
:1042F000983118F0222733274427983028F0232FAD
:10430000342F44279850F9CF992329F046953795B3
:1043100027959A95D9F7912F962742F014D0B0F6A9
:10432000F794E794D7940F5F8BF66ECF10D051F0CF
:1043300008F4CCDEFF2052F2DD0CEE1CFF1C015015
:10434000CBF762CF68CFD20EE31EF41E0895D21AC7
:10435000E30AF40A0895DF92EF92FF920F931F93FE
:10436000D22EE32EF42E052F162F6F915F914F91D1
:104370003F912F910895D895319628F48F938BB75C
:1043800083958BBF8F9100200895F5DFD02CF3DF4C
:10439000E02CF1DFF02CEFDF002D0895ECDF202D75
:1043A000EADF302DE8DF402DE6DF502D089507FBD2
:1043B00000680EF40F7757FB50680EF45F7707FD27
:1043C00002C057FF05C0D216E306F406050708959C
:1043D0002D153E054F055007089500240D280E2881
:1043E0000F28002A0020089591E005C092E003C044
:1043F00094E001C098E028F48F938BB783958BBF2E
:104400008F91B9DF0D929A95E1F7089591E0882395
:1044100021F08894991F8A95E9F7892F909508953E
:10442000883018F011968850FBCF08950181082B31
:104430000183128119231283EF93FF93E2E0F0E0EE
:104440000E949419FF91EF9108950E94A019FF27EF
:104450000E940622EBDFEF93FF93EBE2F5E00E9470
:104460009419FF91EF91182B128309230183EF9385
:10447000FF93E5EFF0E00E949419FF91EF91108116
:10448000182369F4EF93FF93EBE2F5E00E9494198F
:10449000FF91EF911081182311F00E94A319EF935F
:1044A000FF93EBE2F5E00E949419FF91EF910895DC
:1044B0000E940622FF2729915D9148E0B7DFEF9324
:1044C000FF93E2E0F0E00E949419FF91EF9157957D
:1044D00010F4182B1283EF93FF93E2EAF0E00E94AE
:1044E0009419FF91EF91182B1283EF93FF93E2E061
:1044F000F0E00E949419FF91EF914A95F9F62A9500
:10450000D9F608950E940622FF27299148E05527F1
:104510008DDF09230183EF93FF93EDE0F0E00E942C
:104520009419FF91EF9188941081182309F0089451
:104530005795EF93FF93E9E7F0E00E949419FF91FC
:10454000EF914A9529F75D932A9501F708956EDF5B
:1045500009230183EF93FF93EDE0F0E00E949419AB
:10456000FF91EF91E8941081182309F06894EF937C
:10457000FF93E6E8F0E00E949419FF91EF9108950F
:1045800055DFEF93FF93E2E0F0E00E949419FF9172
:10459000EF9116F4182B1283EF93FF93E2EAF0E009
:1045A0000E949419FF91EF91182B1283EF93FF93C0
:1045B000E2E0F0E00E949419FF91EF910895332713
:1045C0003093E6093093E30940DF0EF458C0309190
:1045D000E30930FD54C066276093E5096395609355
:1045E000E40921E050EF48E069DFB1DF31F9AFDFE6
:1045F00032F9632F6670663009F441C0603019F0FB
:1046000031FB40D025C06091E4097091E60967173D
:10461000B1F0C0F48F939F93862F8A95A7EEB9E0EF
:10462000FFDEF4DE7C9178236894772329F4E89404
:104630006091E4096093E5099F918F9109C06894A6
:1046400021D006C0E8941ED06091E4096093E5098A
:1046500097DF6091E40963956093E409613409F0A0
:10466000C4CF6091E5096093E6096623E89409F4F4
:10467000689430F93093E309E89462F808956894F7
:1046800062F808958F939F93A7EEB9E08091E409B3
:104690008A95C6DEBBDE7C9116F4782B01C07923A7
:1046A0007C939F918F9108950F9301E00BBF0F9121
:1046B000889408950F930027F9CF0F9302E0F6CF67
:1046C0000F9303E0F3CF00278A3018F08A50039548
:1046D000FBCF005D0D93805D8D93089580539053C3
:1046E0000027813018F0065F8A95FBCF090F0895E7
:1046F000AF93BF930F939F938F938FB78F93A6E042
:10470000B1E08C9183958D938C3309F03DC088275F
:104710008E9311968C9183958D938C3309F034C0D0
:1047200088278E9311968C9183958D93883161F5AE
:1047300088278E9311968C9183958D939C910EE191
:10474000943089F0963079F0993069F09B3059F0C7
:104750000CE1923039F411969C911197937019F4F1
:10476000039501C00FE1801778F071F081E08E931E
:1047700011968C9183958D938D3031F481E08E93D9
:1047800011968C9183958C938F918FBF8F919F9170
:104790000F91BF91AF91189599278D91939588238B
:1047A000E1F7939511968C9311978E919A95D1F785
:1047B0000895EA2FFB2F00244C918D9103948E32A3
:1047C000E1F711248D9113948823E1F71A941016C0
:1047D00040F41197202F2119239580E38D932A957A
:1047E000E9F7113039F59927AE2FBF2FA00DB91F6A
:1047F000A00FB91F8C919C93853308F421C031E040
:104800008E918E32E9F38D3241F0830F8A3319F4A1
:1048100080E331E001C033278C93AE1789F733234F
:1048200041F0AE2FBF2FB8DF81E34D3209F431964E
:10483000808308958827E00DF81FE00FF81F80831C
:104840000895000F111F221F331F08950095109522
:10485000209530950F5F1F4F2F4F3F4F08950191C7
:1048600010810EC001911191219130810BC00191F5
:10487000108117FF05C03FEF2FEF04C00081112703
:104880002227332737FF03C0E1DF8DE28D93CF93DB
:10489000DF93CF92DF92EF92AA24BB24CC24DD24B5
:1048A000EE2440E2CAE0DD2755E093E38881890FDA
:1048B00087FD9F7083FD907F891B89935A95A9F787
:1048C000C0DFAA1CBB1CCC1CDD1CEE1C4A9551F79A
:1048D000E894EFE0FF2782910ED0EB30E0F71EF076
:1048E00068948A2D0CD088278D93EF90DF90CF901D
:1048F000DF91CF910895982F829501D0892F8F70E5
:10490000805D26F0803309F4089568948D930895AE
:1049100041E003C042E001C044E0E40F8827F81FF3
:104920008291982F829506D0892F04D04A95C1F79D
:104930000C94A1248F708A3008F0895F805D8D937C
:10494000089588278D93089581918D938823E1F7A9
:10495000089594E081918D939A95E1F70895FF93DE
:104960005527F8E0469508F4500F57954795FA9566
:10497000D1F7FF910895FF93881BF9E0001FFA9586
:1049800011F4FF910895881F841B18F4840F8894F4
:10499000F5CF0894F3CFA4DBADDB0395AAF087E154
:1049A000DD0CEE1CFF1C8A9589F00A95CAF7FF20E2
:1049B0005AF000240D280E280F28002039F00A95FF
:1049C000DD0CEE1CFF1CDAF70A95A6CB24CC23CC19
:1049D00087DB0023E2F301DD19F416DC006808959B
:1049E00085E01EDBFF0C001F04830FE70695F7949C
:1049F000FBD0506872DCBBDB139721E438E743ED52
:104A00005BEB2BDC27E831ED43E15DE3D6D02EE014
:104A10003CE343EC5DEBD1D022E83DEA4BE25EE3C0
:104A2000CCD02CEE32E846E75EEBC7D020E931EE81
:104A300049EA5EE3C2D020E83FEE4FEF5EEBBDD027
:104A400024EC3FEF4FE75FE3B8D091DB139784810D
:104A50008F5799F02AF4D82E0FEFE02EF02E04C0D5
:104A6000D82EEE24FF2400275FDB28E132E741E364
:104A70005FE3F3DB3ADB349730DCDFCA31DB80E025
:104A800003C02EDB802F8078882321F0DF92EF9205
:104A9000FF920F938F932EDB802F839512F4BBDB55
:104AA0001BC080958A95885E0AF415C088501AF458
:104AB0000CD0D92210C0DD2488501AF406D0E92287
:104AC0000AC0EE2402D0F92206C09FEF8770990F2A
:104AD0008A95EAF7089520DB8F918823D9F35F91B7
:104AE0004F913F912F910F9362DC0F9199F390F3C7
:104AF0007BD05068F2CB88DBA0CAF2DA86E090DA8D
:104B000005830F772BE33AEA48EB5FE3A6DB2FDB65
:104B1000139741D028F4858188236AF77CDB8DCAFE
:104B20008F778483DDDA349737DF21DB139723E631
:104B300032E446E357EB91DB29ED37EA4AE159E3EA
:104B40003CD026E538E14EEA5AEB37D026E53CE882
:104B50004DE15CE332D02DEC37E543E65DEB2DD043
:104B60002DEE3DEF45E75EE328D028E132E741E353
:104B70005FEB23D039D0B1DBFFDADD24EE24FF2454
:104B800004818FE7080F0695F79411DB8581881F54
:104B900008F4FFDA52CAAEDA8827039512F4889433
:104BA000089507301AF0812F08940895FF1C881F7C
:104BB0000A95E2F7812B889408958FDB96DA349773
:104BC0004CCB0BDC81F00F930F772F933F934F93D8
:104BD0005F93FFDE5F914F913F912F913EDB8EDF20
:104BE0008F918078082B08955FE340E833272227D0
:104BF000089576DA0F930F776ADB44DF8F91807820
:104C0000082B089500000000E17A143E0000A04245
:104C1000000068C20000C6C2000020C197FF1FC18B
:104C200017B7D1B897FF1F41000020410000C642CE
:104C30006F12833A0024744972F97F3F00007A446E
:104C40000000803FF0FF7944E7FB1F417DFFC74232
:104C50000000C8420000F0410000FE420000B442E3
:104C6000CDCCCC3D0AD7A33C14AE073F000090400A
:104C7000CDCC0C41000060410000E040000000008D
:104C80000000F04130392F30342F33300000323300
:104C90003A35383A30300000484F4C442050575293
:104CA0000000425554544F4E0000555342204D4F82
:104CB00044450000504F5745520044533138533259
:104CC000300053455249414C00004E554D4245522B
:104CD000000052454C454153450020642D2020647E
:104CE0002B20206D2D20206D2B20000041444320DF
:104CF000544553540000202020200000524C000056
:104D0000504841534500525353005053322D320006
:104D10005053322D36004443203556002D2D2D2D75
:104D20002D00444320535550504C5900206B2D20EA
:104D3000206B2B20206F2D20206F2B2000002000C7
:104D4000202B00002B0064426D004E4F20494E5036
:104D500055540000206E570020755700206D5700F5
:104D600020572000206B5700202000002053494787
:104D70004E414C2000004D41583620706F776572CF
:104D80006564206279200000555342206F6E6C7973
:104D900020706F77657265640000560020204443E0
:104DA00020737570706C61792020202000002042F3
:104DB00075696C6420696E20414B4B5520200000C2
:104DC000544F204849474800535550504C59000013
:104DD000564F4C5441474500544F204C4F5700000C
:084DE0004241545445525900B0
:00000001FF
